:020000040000FA
:020000007E2858
:080008007A2EC50000300A2821
:10001000C5004030C60045207C304E2046084E20AA
:1000200045084E204A20152008000A30C000182834
:10003000C00B1728080028306626383005203930D4
:1000400005201430052070300520563005206C3016
:100050000520C8306626383005200C3005200130D8
:100060000520013066265926080041208A110A120F
:10007000C40A0319C30A003E031940280820352882
:10008000080043088A0044088200871407140710F8
:10009000871008008714071007140800C7000830ED
:1000A000C8000710C71B071487148710C70DC80B9B
:1000B00051288316071483128714000087108316B3
:1000C0000710831208000830C80083160714831233
:1000D0008714031007180314C70D8710C80B68286E
:1000E000831607108312470808000710871487102B
:1000F00007140800071487148710080083018B0178
:100100008501870107309900831691013F308500F2
:1001100030308700263095002E30960070308F00EA
:1001200008308100831281018B170711071487148F
:1001300063261B200C30052087150230B400803068
:1001400005200030C300E230C4003520C030052057
:10015000352074267426803005203520C0300520D7
:10016000352074267426B40B9F2887110130052092
:1001700074267426A901A917B201B3012E30050512
:100180000C3A0319002E070E0339033AA300031D8E
:10019000CB280530D628023023020318D128093095
:1001A000D628031DD5280630D6281630A8002121D0
:1001B00003302302031DE12802302505A700C030CB
:1001C000A505522946346D34533474346534723481
:1001D00065346F34003452346134643469346F34BC
:1001E0002034493449340034563465347234203470
:1001F00031342E343034373400342034623479349E
:1002000020344D342E3459342034003420345634C4
:100210006F346C343A3420342034203400342034A9
:100220004C34653476343A3420342034203400346D
:100230002A3420345334653465346B3420342A3402
:1002400000342308230723078316263E9B008312CE
:10025000243084000330B40083161C141A089B0A4F
:1002600083128000840AB40B2C290800230823077A
:1002700023078316263E9B0083122430840003301C
:10028000B400000883169A001C1555309D00AA3052
:100290009D009C149C184A299B0A8312840AB40B63
:1002A00041290800A91B5A29A91E652907111B20ED
:1002B0000C300520E621A91B0C24A90129170508EB
:1002C0002E392E3A031D5F297529051DA621851C8F
:1002D000B92129187129851ECC21851DD821A91C79
:1002E0008029E6210C24A9015F268B123C30A20054
:1002F000383081002730A0001030A1008B16522921
:10030000291D8529472429115229A91D942932180C
:1003100091292A08C3002B08C400C03005203520CD
:100320009229B424A9115229291E9929362129126A
:100330005229A91E5229071587110B108B1563002E
:1003400005082E392E3A03199D2952295F260519D1
:10035000B629291403302302031DB029A710B6299A
:10036000A403240A031DB6292808A400051DB629E4
:1003700008005F268518C929291403302302031DAC
:10038000C329A714C929A40A240828020318C929C3
:10039000A401851CC92908005F26851AD529A9143E
:1003A000A603260A031DD529A601851ED529080006
:1003B0005F268519E329A914A60A26080F3C03180D
:1003C000E3290F30A600851DE32908002308031D3B
:1003D000EE290230C3004030C400FD290230230260
:1003E0000318F7290230C300B830C400FD29031DEB
:1003F000212A0330C3008030C4002408B500031054
:10040000B50DB50D3508B600B50D350D0318C30A89
:1004100036070318C30AC4070318C30A803005202F
:1004200035204308AA004408AB000930C40703186C
:10043000C30A4120AC00C40A0319C30A4120AD001D
:10044000282A803005200130C3001830C400352030
:10045000C03005200130C3000630C40035200A300A
:1004600026020318372AC630052026083D2AC53043
:100470000520313008200A302602303808200800D4
:100480004D34493444342D3446344D3420342034F2
:1004900000342034373436342E3431344D3448343B
:1004A0007A340034003458345A34493450342D34BA
:1004B00046344D342034203400342034373437343B
:1004C0002E3438344D3448347A340034043498347B
:1004D00046344D342034413449344334483449346B
:1004E00000342034383430342E3437344D344834EA
:1004F0007A3400340B34D8344E3448344B342034FE
:1005000046344D34203420340034203438343234EE
:100510002E3435344D3448347A3400341034583461
:1005200054344F344B344134493420342034203453
:1005300000342034393432342E3439344D34483494
:100540007A3400342A345834433442344334203427
:1005500020342034203420340034203439343334EF
:100560002E3437344D3448347A3400342C345834F3
:100570004E34413443344B34353420342034203429
:1005800000342034373439342E3435344D34483443
:100590007A3400340834D83454344F344B3459341A
:1005A0004F34203446344D34003420343834303421
:1005B0002E3430344D3448347A3400340A3418340C
:1005C0004A342D34573441345634453420342034A1
:1005D00000342034383431342E3433344D344834FC
:1005E0007A3400340D3458344E3448344B3420348B
:1005F00059344B34483420340034203438343134C6
:100600002E3439344D3448347A3400340E34D834EE
:100610004E3448344B34203454344B344F3420342B
:1006200000342034383432342E3435344D344834A8
:100630007A3400341034583459344F344B344F34F6
:10064000483441344D344134003420343834343467
:100650002E3437344D3448347A3400341534D83499
:1006600049346E3474346534723446344D34203435
:1006700000342034383439342E3437344D3448344F
:100680007A340034223458345434423453342034CD
:1006900046344D342034203400342034393430345E
:1006A0002E3435344D3448347A34003424345834BC
:1006B000423455344E344B344134203446344D3476
:1006C00000342034393431342E3436344D34483407
:1006D0007A340034273418344E344934503450348A
:1006E0004F344E3420342034003420343934333401
:1006F0002E3430344D3448347A3400342A3498342B
:1007000043344F342E3443344F342E344C344F342E
:1007100000342034373436342E3435344D344834B4
:100720007A34003401345834423465344834613406
:100730007034703479342134003420343734383410
:100740002E3439344D3448347A3400340734583434
:1007500046344D3420344F34533441344B344134D7
:1007600000342034383435342E3431344D34483468
:100770007A3400341634D8344E3448344B34203470
:1007800046344D3420342034003420343834383466
:100790002E3431344D3448347A3400341E345834D5
:1007A0004D34423453342034203420342034203427
:1007B00000342034393430342E3436344D34483417
:1007C0007A340034243498344F344234433420345F
:1007D000203420342034203400342034393431346F
:1007E0002E3439344D3448347A3400342734D834F4
:1007F00041344234433420342034203420342034F3
:1008000000342034393433342E3433344D344834C6
:100810007A3400342B345834A91F2E2C4520203034
:100820004E20D0304E2001304E20033023020319D9
:100830001E2C2C084E202D084E20232C24084E2040
:10084000250818384E2000304E2000304E208830C9
:100850004E20260880384E204A20462C291C3F2C4A
:10086000033023020319372C0330DD24462CD1300A
:100870002704AC000130AD000230DD24462C883066
:10088000AC0026088038AD000530DD2408002E308D
:1008900084000A30EC242E1F472C840A0B30EC24F1
:1008A00087112E198715300C7F39B500DF26C0302F
:1008B00005200130C3000F30C4003520C5300520AD
:1008C000383084000230B40000080820840AB40BD9
:1008D000642C0330230203196E2408002E08B6008E
:1008E0002F08B500B60CB50CB60CB50CB60CC03064
:1008F000B6050230C3004030C4002808B4004308E5
:10090000AA004408AB001230C4070318C30A4120F0
:10091000C40A0319C30A3502031D932C4120C039B0
:1009200036020319A22CC40A0319C30AB40B7F2C84
:10093000803005200830B4003F300820B40B9C2CD8
:100940003214AE2C2A08C3002B08C40080300520C6
:1009500035204308AA004408AB0032103508A40033
:1009600036082704A50008003318BC2C2E080339CC
:10097000BC002F08BD00C02C2408BC002508BD0009
:100980000230BE00F830BF00B126B826C0303318A0
:1009900080300520383084000430B40034032E3019
:1009A0000319082000080820840AB40BCE2C02305A
:1009B000C3004E30C40035200800B5002C30840040
:1009C000452022304E2035084E2000084E20840A53
:1009D00000084E204A200800B500452022304E2055
:1009E00035084E20452023304E206320752080009E
:0C09F000840A63207A2080004A2008005E
:100C00002E3005062E39031D002E3314A401A50134
:100C1000A301AC011830AD000230A6000C247426EC
:100C20007426B4244724851E102E051D2F26851CEE
:100C30004226291C132E2408B6002508B500B60C40
:100C4000B50CB60CB50CB60CC030B6053508AC000A
:100C500036081838AD000330DD242910102E5F2629
:100C60000519B0292914A503250A031D3F2EA40345
:100C7000240A031D3F2E0130A4004030A500051DAD
:100C80003F2E08005F268518562E291401302402B5
:100C900003184F2EA50A031D562EA40A562EA50A88
:100CA00041302502031C562EA401A501851C562E99
:100CB00008002730C0005C2EC00B5B2E08001E30E1
:100CC000662E6430662EC830662E0130C100DD30DD
:100CD000C0006A2E6B2E6C2EC00B692E0000702E89
:100CE000712EC10B672E08000A30C2006126C20BAC
:100CF000762E0800F0000308F10083120B19832EF2
:100D00000B18AA2EAC2E0B11383081000130A10235
:100D100003198E2E0318AC2EA002AC2EA008031DC2
:100D2000AC2E2730A0001030A1003B302202031966
:100D30002915393022020319A91537302202031D63
:100D4000A52E291F2916291B2913A20BAC2EA91683
:100D50008B12AC2E0B108B1171088300F00E700EED
:100D600009003F08BD070318BC0A3E08BC0708007D
:100D70003C308400CB26CB26CB26CB26CB2604309A
:100D8000B4000008303C031DCA2E20308000840AC5
:100D9000B40BC12E08001030B400B6010310BD0D15
:100DA000BC0DB60DF63036070318B6000318BD0AA1
:100DB000B40BCE2E84033608303E800008003A3053
:100DC0008400F026F026F0260230B4000008303C03
:100DD000031DEF2E20308000840AB40BE62E08009D
:100DE0000830B400B6010310B50DB60DF630360765
:100DF0000318B6000318B50AB40BF32E84033608A3
:060E0000303E80000800F6
:02400E00C43CB0
:1042000043006F0070007900720069006700680069
:1042100074002000280043002900200032003000F4
:10422000320030002D00320030003200310020001A
:104230006200790020004D002E00590061006D00E1
:1042400061006D006F0074006F00FF00030000004C
:104250000200040000000200030000000200000051
:044260000200020056
:00000001FF
